:020000020000FC
:100000000C94940EC6C10000000000000000000027
:1000100000000000000000000000000000000000E0
:10002000000000002DC000000000000097C000008C
:1000300000000000000000000000000000000000C0
:10004000A0C0000000000000000000000000000050
:100050000000000002030406080C10182030406065
:1000600080000406080C10182030406080A0C000FA
:100070000003070F1F0005050D050205030302001D
:100080004FB662FD0DC0552049F00994C52DC095AD
:10009000089483FDC795C093B20064604FBE189565
:1000A000C0910401089483FDC795C093B2006B7F93
:1000B000C0910401CF3F09F419C04FBE2B982C9872
:1000C0002D9818952B982C982D9876FD0DC065FDD0
:1000D0000BC0C5E0CA95F1F7C0915101C0FD2A9A45
:1000E000C1FD289AC2FD299A4FBE18952092B200F0
:1000F000CC27C160C7BB6460F7CFC8CF70FFC6CF45
:1001000065FDC4CF2B9AC2CF70FFC0CF65FDBECFB7
:100110002C9ABCCF70FFBACF65FDB8CF2D9AB6CF61
:100120002A9870FFB3CF65FDB1CFC1E4CA95F1F74E
:100130002B9AACCF289870FFA9CF65FDA7CFC1E45B
:10014000CA95F1F72C9AA2CF299870FF9FCF65FD31
:100150009DCFC1E4CA95F1F72D9A98CF4FB6C091C3
:100160006F00CD7FC0936F006E7FC0918400CE0D75
:10017000D0918500DF1DD0938900C09388004FBEC9
:1001800018953FB68F7EADB3A170A2118061A0E03B
:10019000ADBBA0916E00AE7FA0936E007894A0914D
:1001A0000801AA2341F085FD2BC0A0910801AA9562
:1001B000A093080125C040E050E085FD15C0A9B11D
:1001C00096FDA095A2FD4FEFA3E096FDA2E0A093BF
:1001D0006900AA27A160ACBB8D7FA9B196FDA0954F
:1001E000A2FD5FEF451739F7A8E161FDA093080173
:1001F00085FD03C0A8E1A09308014093360181600A
:1002000085FD0EC0A0910901AA2331F0A09109013A
:10021000AA95A093090104C08061AA27A160ACBB84
:1002200080FF3DC0A09136014A2F61FF8E7F85FD82
:1002300018C0403F08F040EFA42FA295AF704A0FBE
:1002400050915601533069F0A695A69550FD01C016
:10025000A69552FD03C0A41B4A2F03C04A0F08F401
:100260004FEFA0913F014A1708F44A2F4093010134
:10027000A72FA670A1F073FD12C0A0911001AA0FC4
:10028000AA0F50913E0156955695541708F0452FE8
:100290004A0F4093010118F4AFEFA0930101A09120
:1002A0000101A093030140910301A0913B014A1772
:1002B00008F04A2F542EA0914001AA2309F422C02D
:1002C000542F5A1B10F4A42F50E0BA2E8894AA1F62
:1002D000AA2EA0914201A095AA22A50E58F0A091A5
:1002E0004101A21509F0AA95AA0EA093410148F078
:1002F0004A2D08C0A0914101BA1608F0A395A09319
:1003000041014FEF40930401A52DA03408F068602F
:10031000A0910001A395A093000161F0F894A09131
:100320006E00A160A0936E0084FF02C0A1E0ADBB8F
:100330003FBE1895A0911401A395A093140141E02C
:1003400050910801552329F085FF03C05A95509319
:100350000801A0913601A13018F0209239010DC09A
:1003600020923A0120924301A0913901AF5FA093FE
:10037000390118F0AFEFA0933901F894A0916E0005
:10038000A160A0936E0084FF02C0A1E0ADBB3FBEA0
:1003900018953FB640918400509185008F7EADB393
:1003A000A170A2118061A0E0ADBBA0916E00AE7FF4
:1003B000A0936E00789481FD25C0A2E096FDA3E095
:1003C000A09369008260A9B196FDA095A2FF05C027
:1003D000409305015093060141C1A3E096FDA2E0C0
:1003E000A0936900AA27A160ACBB8D7F85FF01C0E7
:1003F00028C140E0A9B196FDA095A2FD22C140937D
:10040000360111C1A3E096FDA2E0A09369008D7FA3
:1004100061FF72C0A2E096FDA3E0A0936900AA2745
:10042000A160ACBB82604093310150933201A09037
:100430002F014A19B09030015B09BB24A22C4C3823
:10044000520518F42092350149C0A0917401AA23E5
:1004500059F1483C520528F4A0E1BA2EAAE0AA2E90
:1004600023C04836A1E05A0728F4A8E0BA2EAFE02E
:10047000AA2E1AC0403DA2E05A0728F4A4E0BA2EE2
:10048000AEE1AA2E11C0403AA5E05A0728F4A2E036
:10049000BA2EACE3AA2E08C04839A8E05A0720F4C7
:1004A000A1E0BA2EA8E7AA2EC42EA0913301CA1A41
:1004B000D52EA0913401DA0ADD202AF4AFEFC094E2
:1004C000D094CA1ADA0A20923501A8E0A210A0E05E
:1004D000CA14DA0618F4A1E0A09335014093330161
:1004E00050933401409131015091320140932F01DA
:1004F0005093300142E097C0A09105014A1BA091A2
:1005000006015A0B94FD82C093FD80C092FD7CC011
:1005100086FF03C0D52EC42E0CC05695479591FD7D
:1005200073C05695479590FD6FC0D52EC42ED694B6
:10053000C79461FD19C0AC2DAC51AD2DA24008F09F
:1005400005C0DD2089F4AC2DA85C70F4A0910701F2
:10055000A395AA2311F0A0930701AA3008F471C053
:100560002092360181606DC0A0910701AA2319F085
:10057000AA95A0930701A22C50915A0197FD06C09D
:10058000A0906801533011F4A0907001AAEFAA0E58
:10059000A22DA21DCA18DA0A4FB74170533049F490
:1005A000442321F087FD05C0806803C087FF01C098
:1005B0008F77442359F0533031F4AFEFC094D09487
:1005C000CA1ADA0A03C040E050E020C0533049F4B0
:1005D000CC0CDD1CAAE0CA1AD20818F4A0E0CA2E7E
:1005E000D22CAFEFCA16D20418F04FEF50E00EC075
:1005F000A0914C01CA9E412D000C441F50E008F010
:1006000012C04FEF50E00FC05695479594FF07C0BA
:10061000552309F04FEFA42FA6954A0F521D4F3FC7
:10062000520508F04FEF40933601816061FF09C029
:10063000AFE1A095A923AB299A2F8F7DBB2009F4A8
:100640008062A8E1A093080185FF03C0AAE0A093FF
:10065000080161FD03C085FD01C08F7E85FD03C0DB
:10066000A6E0A0930901F894A0916E00A160A09368
:100670006E0084FF02C0A1E0ADBB3FBE189511E043
:100680000AC013E008C01AE006C01EE104C014E668
:1006900002C018EC00C005E1BB27BA95F1F70A9536
:1006A000D9F71A95C1F708952AE338E709C020E37E
:1006B0003CE806C02AE234EB03C025E238EC00C077
:1006C00012E0BB272898BA95F1F72C9ABA95F1F762
:1006D0002C98BA95F1F7289ABA95F1F7123009F0EB
:1006E0002B9A123009F42D9AB0914D01BA95F1F779
:1006F000123009F02B98123009F42D98B7E8BA950A
:10070000F1F71A95F1F6022FB22FBA95F1F70A9583
:10071000D9F73A95A9F628980895221B39E0001FC9
:100720003A9509F40895221F211B18F4210F88948B
:10073000F6CF0894F4CF622C722CB0E08894B39575
:10074000221F331FE0F7379527958894912E802E2E
:10075000020B130B10F4192D082D10F4889401C00E
:100760000894661C771CBA9571F7172D062D08950D
:10077000322D11232AF43A9500951095031B130B83
:10078000F894029F712C002D129F912C802C78944C
:10079000780C172D921C292DB4E06B2E26951795F9
:1007A00007956A94D9F7332321F000951095031B20
:1007B000130B0895089510911B01169500911A01CD
:1007C0000795B0911E01B01B0B2FB0911F01B10B0B
:1007D0001B2F28F40038BFEF1B0740F009C00F376C
:1007E000120508F405C00FE710E002C000E81FEF93
:1007F0000093230110932401089500912301B091E7
:1008000020010B0F10912401B09121011B1F20E04A
:100810003091240133230AF42A95B09122012B1F31
:100820001AF4203F40F00AC02F3008F407C00FEF41
:100830001FEF2FE003C000E010E020EF3091030134
:10084000B0913B013B1718F4323030F009C0B09141
:100850002401BB235AF004C0B0912401BB2332F41D
:1008600000932001109321012093220108952091EB
:10087000770100912301000F10912401111F0E94A4
:10088000B80311232AF40038BFEF1B0740F009C05A
:100890000F37120508F405C00FE710E002C000E8AA
:1008A0001FEF002352F0B0910201B01B0B2F18F084
:1008B000013008F00AC001E008C000950F5FB09158
:1008C00002010B0F08F001C00FEF009325010895FE
:1008D0002091780100912101109122010E94B8031A
:1008E00011232AF40130BFEF1B0740F009C00F3F6E
:1008F000120508F405C00FEF10E002C001E01FEF81
:10090000112352F0B0912501B01B0B2F18F00130CC
:1009100008F00AC001E008C000950F5FB091250102
:100920000B0F08F001C00FEF0093030108950FEFC4
:10093000677F71FD2AC072FD09C06860B0911B011C
:10094000BA3020F0B52DB03408F4677FB091730150
:10095000BB23D9F0B0911B01BB23B9F00FEF10916D
:100960001B010E948D03F894B091130172FDB5E054
:100970000B9F112D002D7894112309F00FEFB091EA
:100980003E010B1710F400913E0100933D010895C4
:1009900000911A0110911B0100541140B0913D01CA
:1009A00010F4BA9501C0B39511F0B0933D010895CC
:1009B00000C0089520915501B0917A00B6FDFACF9C
:1009C0000091780010917900B0917A00BF77B093D0
:1009D0007A00B0914A01B395B0934A01B83060F102
:1009E00020924A01B0917201BB2321F1112329F019
:1009F000B0914B01BF3F61F009C0B0914B010B17A3
:100A000039F020F4BB2321F0BA9502C0B395E1F38D
:100A100000913B01B0934B01B03050F400ECB0308A
:100A200038F400E8B03020F400E4B03008F400E01E
:100A300000933B017F7E0895B0913B01B39511F087
:100A4000B0933B01B0914A01B73009F47061089549
:100A500002E3F894B09179010B9F012D000C001F67
:100A60007894B0913B010B1710F000913B0100937B
:100A7000010100930301502E0093040100933E01F5
:100A8000089520921A01B0EFB0931B010895F894D5
:100A90000091840010918500209114017894309188
:100AA0001501609016010093150110931601031BA8
:100AB000160971FD03C077FD7DC027C07090170136
:100AC000209317012709222311F00FEF1FEF8090C9
:100AD000180190901901309318016092190100914A
:100AE0001501109116010819190920911A01309168
:100AF0001B0136952795020F131F10F40FEF1FEF00
:100B000000931A0110931B0129C020911A01309102
:100B10001B013901B4E08B2EB2E09B2E343010F073
:100B20008A949A94383010F08A949A9476946794C0
:100B30008A94E1F726193709992021F0169507952F
:100B40009A94E1F7200F311F20931A0130931B0173
:100B500028F43FEF30931A0130931B01323008F430
:100B6000706871FF02C0B3E00DC0B09164010091E4
:100B70001101023838F0B395003A08F0B395B63059
:100B800008F0B5E09B2EB4E08B2E10911B01009174
:100B90001A0124E0169507952A95E1F7081912091C
:100BA00028F0B02FB250B12FB20910F402E010E0DB
:100BB000980126C020911A0130911B0139017694C9
:100BC000679466946694669426193209069506958C
:100BD000200F321D20931A0130931B01323008F090
:100BE0007F7704E0369527953695279526952695A7
:100BF000201B10F0223008F422E08901909064015B
:100C000060FDFECFE0902B01F0902C016160B0916F
:100C10006F00B260B0936F00380177FD41C07694E9
:100C2000679400932B0110932C01B92DB330E1F0A0
:100C3000B0FD04C0060D171D930106C0000F111F63
:100C40000250120922E030E0B92DB33068F0209351
:100C50002D0130932E0100932701109328016092FB
:100C6000290170922A013AC000932D0110932E01A0
:100C700020932701309328016092290170922A0164
:100C800071FF0DC0BFE0B0932D0120922E01B093F3
:100C9000290120922A01B0932B0120922C011EC021
:100CA000669400932B01B92DB33091F0B0FD03C0D1
:100CB000060D262D03C0000F025022E0B92DB330DF
:100CC00038F020932D01009327016092290106C07E
:100CD00000932D01209327016092290100911C01AE
:100CE00002FD0350013039F495FD0EC0B5E0B06C43
:100CF000B0937C000DC0023029F4B4E0B06CB09326
:100D00007C0006C095FDF2CFB3E0B06CB0937C00E0
:100D100000914201000F10F4BBE60B270093420143
:100D200060FDFECFB2E0B0930E016160B0916F0044
:100D3000B260B0936F00B72FB67001F120911A0125
:100D400030911B01369527953695279571FF02C086
:100D5000B0E43B0FF8940091840010918500020FDD
:100D6000131F10938900009388006160B2E0B6BB46
:100D7000B0916F00B260B0936F0078940895606195
:100D800020921D0120E067FD20E206C060612092F4
:100D90001D0120E267FD20E001E011E077FD11C0B8
:100DA000B72FB67009F06F7E14E100911B01069514
:100DB00009F403950F3008F00FE071FF02C004E161
:100DC00014E160FD10C0B0911D01BB2361F071FF03
:100DD00006C0B0910E01BA95B0930E0111F4706285
:100DE00052C00E949506B0917B00BF7BB0937B0000
:100DF000B0B7B0917B00B064B0937B00B0911D019F
:100E0000B395B0931D01B0B777FD06C0B1E071FD99
:100E1000B3E0BA95F1F7B0B7B072B21709F028C0D5
:100E200071FF05C00395011708F00A95CACF64FD4C
:100E300005C00395011708F0AFCFC3CF6F7EF894BC
:100E4000309184006090850070901A0180901B01A1
:100E5000370D681C60928900309388006160B2E0B1
:100E6000B6BBB0916F00B260B0936F00789494CF2E
:100E7000B0910D01B13008F48FCF64FD8DCF0A958C
:100E800009F09FCF7F7D20912D0130912E01F894A4
:100E9000B2E0B6BB0091840010918500020F131FD1
:100EA0001093890000938800E0902701F0902801BA
:100EB0006160B0916F00B260B0936F007894B72F0B
:100EC000B67039F0B0910D0172FFB395B0930D017A
:100ED00009C075FF07C067FD05C064FD03C0BF9171
:100EE000BF918DC5089500E063FF03C064FF01C09A
:100EF00001E0F89410911101B7E01B9F212D102DF6
:100F00007894200F26951795269517952695179571
:100F100010931101183718F4B8E7B093110100913C
:100F20001101B09112010B1720F060622B982C98E0
:100F30002D9860FDFECFE0902901F0902A016160BC
:100F4000B0916F00B260B0936F000895B2E095FD6C
:100F50000AC0F894B0931C0128982A9A62FF01C035
:100F60002D9A7894F4C0F894B0931C012898299A8B
:100F700062FF01C02B9A7894EAC0B3E082FF24C0DC
:100F800095FD11C002E0F894B0931C01EAE9F0E08D
:100F9000009351012D98299862FF02C02C9A01C03C
:100FA000289A7894D4C002E0F894B0931C01EAE93E
:100FB000F0E0009351012B982A9862FF02C02C9A0E
:100FC00001C0289A7894C3C095FD0BC0F894B093E3
:100FD0001C01E4E8F0E02D9862FF01C02C9A78949F
:100FE000B6C0F894B0931C01E4E8F0E02B9862FFDF
:100FF00001C02C9A7894ABC0B4E095FD0AC0F89477
:10100000B0931C012A98299A62FF01C02C9A789407
:101010009EC0F894B0931C0129982A9A62FF01C0DF
:101020002C9A789494C0B5E082FF24C095FD11C03D
:1010300001E0F894B0931C01E0E9F0E00093510165
:101040002C98289862FF02C02B9A01C02A9A7894A3
:101050007EC004E0F894B0931C01E4EAF0E0009351
:1010600051012C98289862FF02C02D9A01C0299A3C
:1010700078946DC095FD0BC0F894B0931C01EEE719
:10108000F0E02C9862FF01C02B9A789460C0F8942D
:10109000B0931C01EAE8F0E02C9862FF01C02D9AA1
:1010A000789455C0B6E095FD0AC0F894B0931C0141
:1010B0002998289A62FF01C02B9A789448C0F89426
:1010C000B0931C012A98289A62FF01C02D9A789447
:1010D0003EC0B1E082FF24C095FD11C004E0F89449
:1010E000B0931C01E4EAF0E0009351012B982A9898
:1010F00062FF02C02D9A01C0299A789428C001E0AD
:10110000F894B0931C01E0E9F0E0009351012D98B0
:10111000299862FF02C02B9A01C02A9A789417C0BE
:1011200095FD0BC0F894B0931C01EAE8F0E02B9811
:1011300062FF01C02D9A78940AC0F894B0931C0104
:10114000EEE7F0E02D9862FF01C02B9A78946F7D56
:1011500008952DE730E0F901209251012B982C9849
:101160002D982A98289829986B7F0895A2E5B1E0D8
:101170000FEF0D930D930D930D9303E00D9304E08A
:101180000D930BE00D9301E00D9301E00D9301E051
:101190000D93AEE5B1E001E00D930FEF0D930D93CC
:1011A0000D930D930D9303E00D930FEF0D930FEF40
:1011B0000D930D9305E20D9300ED0D930AEF0D9342
:1011C0000AEF0D9304E00D930FEF0D9301E00D93E3
:1011D00000E00D930AE70D930FEF0D9300E00D93E0
:1011E00001E00D9300E00D9303E00D9300E00D93FB
:1011F0000895209159018B7FB0915A01B33019F0B5
:101200009F7DB1FD90629F7BB0915B01B1FD9064C9
:10121000223011F0886001C0877F08950A95E00FA1
:10122000F21DB4910895E4E5F0E0009152010E94AE
:101230000E09B0937701E4E5F0E0009153010E94BC
:101240000E09B0937801E2E6F0E0009158010E94A7
:101250000E09B093790100915801023008F402E0C0
:1012600000931301B0916E010FEFB23009F400EA60
:10127000B33009F402E800931201E0E7F0E00091D6
:1012800075010E940E09B0934001089508952091C0
:10129000680130916901B0915A01B33009F43E50B0
:1012A00097FF02C020E03FEFB32FB21B6B2EB25866
:1012B00010F4B2E86B2E00E00395609EB12DBD578F
:1012C000D8F300934C01089590680E9447090E944A
:1012D000450320E030E0B0E16B2E0E944103B09165
:1012E00036012B0F321D6A94C1F7B4E0369527956D
:1012F000BA95E1F7822E9F770E9447090895F894E6
:10130000E3E0F0E0B9E0B7BFB491B078C1F3F8948E
:10131000A895B4B7B070B4BFB0916000B861B09395
:101320006000B0E0B0936000B4E0BEBFBFEFBDBFEF
:101330000E94A908B0E0B5B9BFE3B4B9B0E0B8B94C
:10134000B0E0B7B9B0E0BBB9B0E0BAB92224A0E0D0
:10135000B0E02D92AA31E9F7A0E0B1E00FEF2D92B5
:101360000A95E9F7B1E0B09342010E94B6080E94E5
:10137000420DB0E0B06CB0937C00B0917A00B460E4
:10138000B068B0937A0000916A0100934D01B1E01A
:10139000B0930A01F8940E9449030E9454030E94EA
:1013A00045030E9457030E9445030E945A030E946E
:1013B00045030E94D70D0E9449030E9449030E94E1
:1013C0004703F8940AEF1AEFA9B196FDA095A2FF82
:1013D0001FC01A95C9F70A95B1F7E0E0FCE3B59193
:1013E000B43E39F4B591B03E21F4B591BF3F09F454
:1013F0000CC0E0E0F395F395B591B83F49F4B59191
:10140000B43931F4B591BA3A19F4EE27F695099446
:101410000E94F9080E9413090E9446090E94470988
:1014200000916A0100934D010E94A908B2E0B5BD88
:10143000B2E0B0938100B2E0B093B100B1E0B5BBCF
:10144000B0936E00B2E0B6BBB0936F00B1E0B7BB33
:10145000B0937000B0917B00BF7BB0937B00B0B7BE
:10146000B0917B00B064B0937B000E943F037894FE
:101470000E94D80420921001B3E096FDB2E0B09330
:101480006900B1E0BDBBBB27B160BCBB8D7F0E94D2
:101490004903626033E02CE0B0913501BB2321F4B5
:1014A0002CE03A9509F48DCF0E94450380FF89CF47
:1014B0008E7FB0913601B23070F3B92FBF710091B9
:1014C000380100933701B0933801B01721F72A95FE
:1014D00019F76D7FB3E096FDB2E0B0936900BB27CA
:1014E000B160BCBB8D7FB0917401BB2321F48062DD
:1014F000B92FB0709B2F8F7B209207010E9447036A
:1015000085FF05C0B0910701BA3008F080640E94E1
:10151000410302E085FF01C000E0B0913601B01741
:10152000B0F3F8940E9454030E9454030E945403A1
:1015300078940E94490320922601B0915A01B33059
:1015400009F491C00E944103B0915E01B13008F4EA
:101550008AC0B0910A01B13008F485C085FD1EC073
:10156000B0913601BF3F08F47EC0F8940E945D033D
:1015700078940E944703B0913601B130B0F7F894E7
:101580000E9454030E9443030E94540378940E94D3
:101590004703B0913601BF3F90F35EC3B8E09B2E86
:1015A0009068F8940E94470978940E944703F89441
:1015B0009F770E94470980903601B0913601BF376E
:1015C000789408F458C00E943F03F8940E945D0389
:1015D00078949A9429F70E946409B82DB550B09375
:1015E00069010E944903F8940E94750D0E94DD0D67
:1015F0007894BAE09B2E9068F8940E9447097894FA
:101600000E944703F8949F770E9447098090360113
:10161000B0913601BF37789460F70E943F03F89489
:101620000E9454030E9443030E94540378949A94A6
:1016300011F70E946409B82DBB5FB09368010E9446
:101640004903F8940E94750D0E94FA0D78940E9447
:101650004703F8940E9447097894B0913601BF3F40
:1016600008F47CCFF9C200913601B09126010B1726
:1016700010F0009326010E94470301E0B0915A0147
:10168000B35009F405E0B0913601B01708F055CF1A
:10169000F8940E945D030E945D030E945D037894AC
:1016A0000E94490320920A0120920B0120920C0112
:1016B000B0910B01B395B0930B01BF3F91F5B09181
:1016C0000C01B395B0930C01B0916C0109E1BA958E
:1016D00059F002E3BA9541F00DE7BA9529F00AEF07
:1016E000BA9511F020920C01B0910C01B017C8F01E
:1016F0000E94A9080E943F03B0910C01BA95B093D3
:101700000C0120920B01B0916B01B0934D01F89444
:101710000E945D037894B0916A01B0934D010E94DC
:1017200047030E944303B0910801BB2319F485FFCE
:1017300001C047CE01E085FD01C006E0B091360151
:10174000B01708F4B5CFB0915A01B35011F00E9410
:101750004703B0910801BB2309F433CEF8940E94EB
:10176000A908209201012092020120920301522C2B
:1017700020920401209241017894B0915701BB0F4F
:10178000B0933F0120921E0120921F012092200160
:10179000209221012092220120924A0160E070E013
:1017A00020921101B8E0B0934A0170610E943F039A
:1017B000B0E074FDB0E0B06CB0937C00B0917A0002
:1017C000B068B064B0937A00B0917A00B6FDFCCFF7
:1017D0000091780010917900B0917A00BF77B093B2
:1017E0007A00112309F00FEF00934B010E94DA04F5
:1017F000B8E0B0934A0170610E94F908F894BFEF15
:10180000B0933B010E942805B0910101B0933B01C8
:10181000B0933C01B0933D017894B1E0B0930101E5
:10182000B09303015B2EB0930401B0934401B091D7
:101830003A01B0934301B0915A01B33019F49F7D3E
:1018400087FD90627160726020920D010E945208C3
:101850000E9469080E9441050E9447050E944105B7
:101860000E9447050E9441050E94C6060E94DA03B5
:101870000E9473070E94A6070E9447050E94BF06A8
:1018800066FD0E94DB0377FF0E94970477FD0E94AC
:10189000C8040E9473070E94BD070E9447050E946A
:1018A000C60666FD0E94FD030E9473070E94FC07A6
:1018B0000E9447050E94BF0666FD0E9437040E94F1
:1018C00073070E9413080E9447050E94C60666FD22
:1018D0000E9468040E9473070E9452080E944705F4
:1018E0000E94BF06B0E074FDB0E0B06CB0937C0025
:1018F000B0917A00B068B064B0937A000E94730728
:101900000E9469080E9447050E94DA0471FF21C005
:10191000B0913E01B0933B01B0933C01B0913A01CC
:10192000B0934301B1E0B093440118E12CE0B091D1
:101930000D01B11740F07D7F746020930F01BFEF60
:10194000B0933B0106C0B0913601B13008F08CCFA6
:1019500060C072FF11C067FD0FC0B0910F01BA9552
:1019600019F47B7F786080CFB0930F01B09136017E
:10197000B13008F079CF4DC020921001B0913901FB
:1019800002E810917601112309F003E0B01708F086
:1019900040C085FF04C0B0910801BB23D1F1B091D4
:1019A0005A01B33081F495FD03C087FD04C00BC01C
:1019B00087FF01C008C067FD06C06068B0913E01A6
:1019C000B0933B0177CF00EF67FF05C0B0913E01B8
:1019D000B0933B0100E2B0911B01B01708F444CF73
:1019E00067FF17C06F779F7D87FD90627460B2E1DB
:1019F000B0930F01B0913E01B0933B0135CFB09150
:101A00001001B395B0931001B0913601BB2309F0DA
:101A100002C020921001F8940E94A90880905901F8
:101A2000B2E0B09359010E94F908809259012092C6
:101A300001012092020120920301522C2092040104
:101A400020923F0160E070E078940E9447030E947A
:101A5000A90800917601002319F02B9A2C9A2D9A4F
:101A6000B0E0B06CB0937C00B0917A00B460B06824
:101A7000B0937A0085FF05C0B0911001B43008F032
:101A8000A0CC12CEEDE0F0E00E946E0D0A3509F018
:101A90001EC0EEE0F0E00E946E0D053A09F017C09E
:101AA0003AE0A2E5B1E0E3E0F0E00E946E0D0D93B4
:101AB00031963A95D1F739E1AEE5B1E0EFE0F0E0EB
:101AC0000E946E0D0D9331963A95D1F704C00E9495
:101AD000B6080E94750DE8E2F0E00895F999FECF8E
:101AE000E1BDF2BDF89A00B508950E94980D3AE064
:101AF000A2E5B1E0E3E0F0E00D910E94900D319697
:101B00003A95D1F739E1AEE5B1E0EFE0F0E00D91C3
:101B10000E94900D31963A95D1F70E94A30D089539
:101B2000F999FECF00BDE1BDF2BDFA9AF99A089588
:101B3000EDE0F0E00FEF0E94900DEEE0F0E00FEF2F
:101B40000E94900D0895EDE0F0E00AE50E94900DEE
:101B5000EEE0F0E005EA0E94900D089530914E010C
:101B600000914F01313011F400935601323011F4DD
:101B700000935701333011F400935801343011F4BD
:101B800000936401353011F400935901363011F49B
:101B900000937501373011F400936E01383011F461
:101BA00000935A01393011F400935B01089525E048
:101BB0000E9449032A95E1F708950E9454030E9468
:101BC00057030E945A030E945D030E9443030E9430
:101BD00054030E9457030E945A030E945D030E940F
:101BE00043030E9454030E9457030E945A030E9419
:101BF0005D0308950E945D030E945A030E945703EB
:101C00000E9454030E9443030E945D030E945A03F2
:101C10000E9457030E9454030E9443030E945D03E5
:101C20000E945A030E9457030E9454030895809013
:101C30004E0190904F010E9454030E9454030E9451
:101C400054030E9443038A94B1F70E945D030E94EB
:101C500043039A94D1F70895F8940E94DD0D789487
:101C60000E94D70D0E94D70DB1E0B0934E01B1E0B4
:101C7000B0934F0120925001F8940E94170E78946F
:101C8000B5E06B2E709036010E944903B091360189
:101C90007B16C1F7B13018F0BF3F70F10CC00E9445
:101CA000AE0DF8940E94750D0E94DD0DB8E0B09362
:101CB00060000E94D70D6A9429F7B0915001B39546
:101CC000B0935001B33008F4D7CF0E94D70DB09134
:101CD0004F01B395B0934F01F894B0914E01BA956E
:101CE000E6E7F0E0EB0FF21D049178940395B091D4
:101CF0004F01B01708F4BECF0E94D70D0E94D70D38
:101D0000B0914E01B395B0934E01B0914E01BA30EF
:101D100008F4ADCF0E94B608F8940E94750DB8E0A3
:0A1D2000B09360000E94D70DEACADC
:00000001FF
